:020000040000FA
:100000008316FF23900000308500831285011221A2
:10001000122164211221642112216421042104216E
:100020006421122164211221642104216421E2202F
:10003000E22064212321232164212321642123211F
:1000400064213B213B21642123216421122164216D
:1000500023216421122164210421642104216421CB
:100060001221122164216421F0206421F0206421F6
:10007000F0206421F0206421F0206421122112215B
:100080006421F0206421E2206421F0206421E22038
:100090006421D1206421D120D1206421E220E220FA
:1000A00064216421232164212321642123216421EB
:1000B000232164213B2164213B21642123216421EC
:1000C000122164212321642112216421042164214D
:1000D000042164211221122164216421F020642171
:1000E000F0206421F0206421F02064211221642199
:1000F00012216421F0206421E2206421F020642197
:10010000E2206421D1206421D1206421E220E22078
:1001100064216421122164211221642112216421AD
:1001200012216421122164211221642112216421EF
:1001300004216421122164211221642112216421ED
:1001400004216421D1206421D1206421E220E22015
:1001500064216421D1206421E2206421F020642103
:1001600004216421122164212321642112216421AC
:10017000232164213B213B216421532164213B2124
:10018000642123212321642112216421122164216D
:1001900004216421E220E220E22064216421642120
:1001A00007282930AE0005156F218A219421A3214B
:1001B000AD2105116F218A219421A821AD21AE0B1B
:1001C000D32808002E30AE0005156F219421A321FD
:1001D000A82105116F219421A821AE0BE428080065
:1001E0003130AE0005157A2185218A218F21992190
:1001F000A32105117A2185218A2194219E21A821FC
:10020000AD21AE0BF22808003730AE0005157A217B
:1002100085218A2105117A2185218A21AD21AE0B04
:10022000062908003E30AE0005157A21852194216B
:10023000A821AD2105117A2185219421A821AD2184
:10024000AE0B142908004230AE0005157A218A2130
:100250008F2199219E21A321A821A821AD2105113B
:100260007A218A2199219E21A321A821A821AD21AB
:10027000AE0B252908004E30AE0005157A219421D9
:1002800099219E21A321A821A821A82105117A2125
:10029000942199219E21A321A821A821A821A82148
:1002A000AE0B3D2908005830AE0005157A21942187
:1002B0009921A821AD2105117A2194219921A82104
:1002C000AD21AE0B552908001430AE007A218521EE
:1002D0008A218F2194219E21AE0B662908000430CB
:1002E000A100FF30A200A20B73290000A10B71290D
:1002F000000008000230A300FF30A400A40B7E29F8
:100300000000A30B7C2900000800FF30A500A50B0E
:10031000872908008030A600A60B8C2908008030B1
:10032000A700A70B912908002030A800A80B962948
:1003300008001030A900A90B9B2908000830AA006A
:10034000AA0BA02908000830AB00AB0BA5290800B8
:100350000230AC00AC0BAA2908000130AD00AD0B97
:04036000AF290800B9
:02400E00943FDD
:00000001FF
